:10000000830100308A003B28E50003088301E400F7
:100010002B088100AA0AAC0A00308A002C081F397C
:10002000142086000B1135288207083409340A345D
:100030000C340D340E340E340F340F340F340E34B0
:100040000E340D340C340A340934083406340534C3
:1000500003340234013401340034003400340134F8
:1000600001340234033405340634831264088300F7
:10007000E50E650E090022308400593051202030F1
:1000800084002230512083010730E300F730E20082
:1000900059308400623055208301442D04068001CC
:1000A000840A0406031D4E280034F00060208000FE
:1000B000840A040870060319003456288312E200EB
:1000C000E31B6B28631B732863088A006208E20A3B
:1000D0000319E30A82008313631883176208E20A94
:1000E0008400000808008207F6348234A8346034A3
:0800F00084346834FA34003452
:1004180083121D232C3A8312031908000D2A8B120C
:1004280083169B001C141A088B1683120800F00010
:100438000030711870070310F00D0310F10CF1086B
:10044800031908001D2A362A4830D5002E2A83129F
:10045800560879228312D50A55031322D600D608E6
:10046800031D2B2A83120800F401F5010310F30C75
:10047800F20C031C462A7008F40771080318710A65
:10048800F5070310F00DF10D720873040319003419
:100498003A2A3030DA00DB00D50083125A08D90036
:1004A8005B08DA005508DB001D23D5002E3A031936
:1004B800612A55082C3A031D512A8312080030304E
:1004C800DD00DE00D50083125D08DC005E08DD007B
:1004D8005508DE001D23D5002E3A0319772A550842
:1004E8002C3A031D672A831208008511A118851567
:1004F8008312D8000A30D7005130B000211C882A56
:100508005A30B007B00B862A64008312581C912A0F
:100518008515A11C952A8511952A8511A11C952A56
:10052800851503148312D80CD70B802A0800D5012F
:10053800D601D701D800B42A0A30F200F3015608D0
:10054800F1005508F00038225708580784000008C1
:100558000F397407D50075080318750AD600D70A2D
:10056800033083125702031CA02A5608F1005508CD
:10057800F00008001D23BB001D23BC001D23BD0087
:100588001D23BE001D23BF001D23C0001D23C10065
:100598000C221D23C2001D231D23C3001D23C400DC
:1005A8001D23C5001D23C6001D23C7001D23C80029
:1005B8001D23C9001D23CA000C221D23CB00831252
:1005C800080041307922543079220B3079220430E6
:1005D8007922FF300F2B1D23D50083169C18F22A91
:1005E8008312550883169B0083121D2383169A00D5
:1005F80003108B1B03148B1383161C1555309D0099
:10060800AA309D009C141C1103188B179C180A2BE8
:10061800831255081322792283121D23D500573AD5
:100628000319EF2A83125508523A031D08001D23A7
:100638000E2B242B6400061E232B0510252B0514D6
:100648008312051A292BA1181E2B051E2D2BA11C60
:100658001E2BD6011E30B000B00B302B0830D7004F
:10066800640051308312B000211C3E2B5A30B00771
:10067800B00B3C2B03108312D60CA11C462B051A79
:10068800492B482B051E492BD617D70B342B513035
:10069800B000211C542B5A30B007B00B512B8312D9
:1006A800560808006400D701D800083057028312A2
:1006B80003180800A0135818A0170310201F792B3F
:1006C800A80CA90CA01F6A2B01306B2B0030F0007E
:1006D800031C702B0130712B0030F0060319782BA6
:1006E8008430A8060830A90603108312D80C211EEE
:1006F800822B20302A020318862B7D2B3A302A02BF
:10070800031C822BAA01A01F9C2BAE0AA11DA52B9E
:100718002E08053A031DA52B211E972B20302A02EF
:1007280003189B2B922B3A302A02031C972BAA0101
:10073800211AA02BC930A12BE630AB001030A1063E
:10074800AE01D70A08305702031808005E2B061FAF
:1007580005148312D501B72BD601B42B6400D60A31
:10076800560FB22BD50A550FB02BD501D50A031950
:10077800CF2B6400061E061FC52BD501D50A05140C
:10078800C82B061FC82B0510D601203056020318A7
:10079800BA2BD60AC92B1B301322F000701CD62B9B
:1007A8002014D82B831220101B3083121322F00040
:1007B8007019A01CE12B2016E32B83122012831240
:1007C800DF035F0FEB2B16301322DF008312DF08E5
:1007D800031DF92B20301322F000F01B20102130CC
:1007E80083121322F000F01B2012153083121322FB
:0807F800F000700F022C033029
:10080000AD000C2C1530831213222D06031D0A2C6B
:10081000AD010C2C8312AD0A831205152116831627
:1008200081158112C930831281008B17FF30A90016
:10083000A80020131D301322D5008312D5087E3066
:100840000319252C5623D5031D2C56232017A1153B
:10085000AE01D501831255081322D600D50A5508DA
:100860000E3A031D372CAD08031D372CD60A831210
:100870005608562355080E3A03194D2C2A2CD50A32
:1008800055031322D6005508153A031D4A2C2D0B8B
:100890004A2CD60A83125608562383125508153A55
:1008A0000319562C01302D0203183F2C02302D0263
:1008B000031C632CAE3056239230562388305623C7
:1008C0008A30562383122D08023A031D6E2C6430A1
:1008D0005623403056236330562383122D08033AA3
:1008E000031D792C6430562340305623653056233F
:1008F00083122D08043A031D842C663056234030A1
:1009000056236730562383122D08053A031D8E2C7B
:100910006830562340305623693056230330831203
:100920005623F0305623211DBB2C3E305623D501D3
:1009300000308A0083125508732000380319AC2C4C
:1009400000308A008312D50A55037320F00003108B
:10095000700C83125623982C80308312D500D50A50
:1009600055031322D600D60883120319312D5608D9
:1009700056238312AF2C213083125623D501083021
:1009800055020318CB2C831255083B3E8400000807
:100990005623D50ABF2C1E30831213225623D501AD
:1009A000093055020318DC2C83125508433E84009D
:1009B00000085623D50AD02C1F3083121322562349
:1009C000201C022DD501033055020318EF2C831291
:1009D0005508593E840000085623D50AE32C2F30D1
:1009E00083125623D501033055020318022D8312BA
:1009F00055085C3E840000085623D50A0330550292
:100A0000031CF72C8312201E1D2D2F30562341303E
:100A100056233D3056232708303E56232608303EC5
:100A200056232508303E56232408303E56232308FB
:100A3000303E56232208303E562320308312D50004
:100A4000262D831256087F3956238312D50A550363
:100A50001322D600D6080319302DDF080319212DE3
:100A600083122013FF30A906A80629085623280858
:100A70005623A1117E3056237E30562305118B1349
:100A8000061F0510831208000830D300D40164004B
:100A90008B018B1607309F0083168113F030860080
:100AA0001030850083120510851405110530D10022
:100AB000D2012114A114D001D00A6400831252087B
:100AC0005104031D792D2115AB2321115308D100A9
:100AD0005408D2000310D30DD40D0730540209304E
:100AE00003195302031C782D0830D3000730D400BB
:100AF0008312CF0F812D0230A106A11C812D013060
:100B0000A1061D23CC00243A03198C2D4C08213A50
:100B1000031D5D2DE5225D2D83121D23473A031D24
:100B20005D2D83121D23503A031D5D2D8312861AFD
:100B30009A2DA016CF01D0080319A02D27228312C9
:100B4000D0011D23CC00563A03192019B02D1D23C6
:100B5000543A031D5D2D1D23473A0319652F5D2D62
:100B600083124C08473A031DBE2D1D23473A031D2F
:100B70005D2D1D23413A0319C72E5D2D4C08523AB5
:100B8000031D5D2D1D234D3A031D5D2D1D23433A8D
:100B9000031D5D2D83122015023085061D23D1080B
:100BA0000319D203D103B90A0319BA0A0C221D236F
:100BB000563A0319E12E831285141D23BE221D23EC
:100BC00063220C224D221C30831213220038031999
:100BD000FB2D3C30F200F3011C301322F000F10138
:100BE000382275083A02031DF72D74083902031CD8
:100BF000BF2EA016BF2E5C3083129B227008B70058
:100C00007108B80059309B227008B5007108B60011
:100C100019301322F000F1017108803AF20038080F
:100C2000803A7202031D162E37087002031C282E0C
:100C30003C308312F200F30118301322F000F1016E
:100C400038227408B3007508B400B101B2019B2EBC
:100C500014308312AF001A301322F000F101710832
:100C6000803AF2003808803A7202031D392E3708A4
:100C700070020318412E173083121322B300B401FF
:100C8000632E1A3083121322F200F301173013225D
:100C9000F000F10138227408F0007508F1003808FE
:100CA000F3003708F20072277408B3007508B40027
:100CB0003808F3003708F200FA30F0000030F10194
:100CC00072277408AF07513083122F02031C6A2E5B
:100CD0005030AF00600A0319610A031D732E3508F6
:100CE000E0003608E10060083502B1006108031C2D
:100CF000610A3602B200B21F852E35086002B100CB
:100D00003608031C360A6102B2003208803AF0004D
:100D100080307002B53003193102031C9C2E6830FC
:100D2000F0000130F10031087002B1003208031CFC
:100D3000320A7102B20083122F08F000F10171082B
:100D4000803AF2003208803A7202031DA92E31085F
:100D500070020318B22E00303A020630031939022D
:100D60000318BA2E3A083402031DB82E390833028C
:100D70000318C02EA0163508E0003608E1008312E3
:100D8000A01E5D2DAB23A012B901BA015D2D831207
:100D9000A014023085061D232019D52ED108031971
:100DA000D203D103B90A0319BA0A83120C22BE2254
:100DB0001D231D23303A0319E12E3B082C3A031D55
:100DC000E32E85105D2D831285141D230C220C2229
:100DD000A201A301A401A501A601A7011D23CD0025
:100DE000CC012D3A0319E32D83122608A70025080C
:100DF000A6002408A5002308A4002208A30021308F
:100E0000F1004D08D03E1B22CE00643083124E020A
:100E1000031C2A2F9C30CE07A30A0A302302031C8E
:100E2000052FF630A307A40A0A302402031C052F5D
:100E3000F630A407A50A0A302502031C052FF63058
:100E4000A507A60A0A302602031C282FF630A6079B
:100E5000A70A052F0A30F1004E0887274C07A20089
:100E60000A302202031C532FF630A207A30A0A30CD
:100E70002302031C532FF630A307A40A0A302402CE
:100E8000031C532FF630A407A50A0A302502031CC1
:100E9000532FF630A507A60A0A302602031C532F4B
:100EA000F630A607A70A83124E08CC000A304C027F
:100EB000031C5D2FF630CC07562F1D23CD002C3A96
:100EC0000319E32D4D082E3AF22E8312A0151D238F
:100ED0004D2283121D234D3A8312031D6A2F1D23B9
:100EE0006322E32DF601F11F7C2FF009F00A0319AC
:100EF000F103F1097617F61773088039F606F31F28
:100F0000BE2FF209F20A0319F303F309BE2FF00012
:100F1000F4010310FD307107031CAE2FF301F03014
:100F20007105031D962F0430F300F10EF20103103A
:100F3000F30AF10D031C982FF10C710870020318CD
:100F4000F000F20DF30B9C2FF41FA82FF209F20A08
:100F50007208F41F0800F009F00A0800F10C0318E9
:100F6000B72FF10C031CF0010310F00C031C03104D
:100F70007008F200F001F00DA42FF601F401F50164
:100F800072087304031DC72FF001F10100341F30F4
:100F9000F6040310F60AF20DF30D031CCA2FF30C2E
:100FA000F20C73087102031DD72F72087002031C24
:100FB000DF2F7208F0027308031C730AF102F40DAC
:100FC000F50DF60BF61ACF2FF61FEB2FF409F40AE6
:100FD0000319F503F5097408F2007508F300761F8C
:100FE0000034F009F00A0319F103F1090034303438
:100FF000303430343034303430340134FF34FF3462
:02400E00663F0B
:104200008200A0008A00A400B000A20060009C0010
:104210009E0086008200980098006000A4008A003A
:1042200098008200B20040006000030002005A00C3
:10423000140003003200010000003C002F003E008B
:10424000000000000000000000000000000000006E
:10425000000000000000000000000000000000005E
:10426000000000000000000000000000000000004E
:10427000000000000000000000000000000000003E
:10428000000000000000000000000000000000002E
:10429000000000000000000000000000000000001E
:1042A000000000000000000000000000000000000E
:1042B00000000000000000000000000000000000FE
:1042C00000000000000000000000000000000000EE
:1042D00000000000000000000000000000000000DE
:1042E00000000000000000000000000000000000CE
:1042F00000000000000000000000000000000000BE
:10430000610070007200730074007200610063004D
:104310006B00650072002D0030002E00310031006E
:104320002D003100360066003600340038000000F1
:00000001FF
